:020000040000FA
:04000000CB303A289F
:08000800A000030EA100831209
:1000100005191028831601178312B23081002B288E
:1000200083160113831203140B190310A80DA90DD5
:10003000AA0DAB0DAC0DAC16FF302C02031D2B2806
:10004000FA302B02031D2B2831152A08AF0029088E
:10005000AE002808AD008B100B11210E8300A00EFE
:04006000200E090065
:0C007400203084008001840A80300402E7
:10008000031C3C281230B000E02183160C3085059B
:1000900087018312850187010730990000309A009B
:1000A000103083168E008312603083168F00831207
:1000B0000030831691009F008312C83083168100A0
:1000C000831231309000003083168C008312103080
:1000D0008B00831600309B001C141A088312BC008E
:1000E000851DDE22831610309B001C141A08831213
:1000F000BD00831630309B001C141A088312DE00EA
:10010000C52281018E018F010B118B100B108C0108
:100110008B17982031199B20B30B96280310851953
:100120000314B90DF030390203194421042389283E
:1001300064003210080031110130B7008B132030F9
:10014000370783169B001C141A088312A400103072
:10015000370783169B001C141A088312A300A600FD
:100160000230A6060030370783169B001C141A08BD
:100170008312A200A7000130A7068B17321CC628E5
:1001800022090339A200A309A409A50924082F0202
:10019000031D3E2923082E02031D3E2922082D029D
:1001A000031D3E2901303702031DDB283D18DB28E3
:1001B0003D143E14ED2102303702031DE428BD1822
:1001C000E428BD143E14F92103303702031DED2845
:1001D0003D19ED283D153E14052204303702031D5C
:1001E000F628BD19F628BD153E1411220530370238
:1001F000031DFF283D1AFF283D163E141D22063020
:100200003702031D0829BD1A0829BD163E142C22E9
:1002100007303702031D11293D1B11293D173E14DC
:100220003E2208303702031D1A29BD1B1A29BD17AB
:100230003E14492209303702031D23295E18232961
:100240005E143E1454220A303702031D2C29DE1896
:100250002C29DE143E145F220B303702031D352992
:100260005E1935295E153E146A220C303702031DD3
:100270003E29DE193E29DE153E147822B70A0D30DC
:100280003702031808009E280130B600B300B400FE
:10029000B500B70085018701B1139820B30B8C29F5
:1002A000031085190314B90DF03039020319B3296D
:1002B000B40B8C290130370203198922023037022E
:1002C00003198E22033037020319932204303702B8
:1002D000031998220530370203199D220630370290
:1002E0000319A222073037020319A7220830370268
:1002F0000319AC22093037020319B1220A30370240
:100300000319B6220B3037020319BB220C30370217
:100310000319C0229630B400311D4D293111321C11
:1003200096292D090339AD00AE09AF092F1C4D29BF
:100330008E018F010C1C4D290C102E1E4D298B1384
:1003400020303707BB002F08BA00CB211030370709
:10035000BB002E08BA00CB2100303707BB002D08A8
:10036000BA00CB218B1785018701B70AB6010D3082
:100370003702031C4D29C52208003E1C08003E1010
:100380001030BB003D08BA00CB213030BB005E0806
:10039000BA00CB2108008B133A0883161C159A006B
:1003A00083123B0883169B0055309D00AA309D00A8
:1003B0009C1464009C18D9291C1183128B17080007
:1003C000FF30C800CA15CB15CC15CD15CE15CF15ED
:1003D000D015D115D215D3150800C130BD05FF3099
:1003E000DE050130C405C0000030C200C6005F1049
:1003F0000800C230BD05FF30DE050230C405C00074
:100400000030C200C6005F100800C430BD05FF30D8
:10041000DE050630C405C0000030C200C6005F1013
:100420000800C830BD05FF30DE050A30C405C00035
:100430000030C200C6005F100800D030BD05FF309C
:10044000DE053C181030BC181130C405C000003067
:10045000C200C6005F100800E030BD05FF30DE05B9
:100460003C181830BC181930C405C0001830C20040
:10047000C6005F105F17C411441208007F30BD052D
:10048000C030DE050830C505C1000030C300C7001C
:100490000800BF30BD05C030DE051030C505C10005
:1004A0000030C300C70008003F30BD05C130DE0585
:1004B0003030C505C1000030C300C70008003F3020
:1004C000BD05C230DE055030C505C1000030C30097
:1004D000C70008003F30BD05C430DE053C18803041
:1004E000BC188830C505C1000030C300C700080033
:1004F0003F30BD05C830DE053C18C030BC18C830E0
:10050000C505C100C030C300C700DF174513C513C0
:100510000800103085060030870608002030850668
:100520000030870608002130850600308706080065
:10053000223085060030870608000030850602302C
:100540008706080002308506023087060800003062
:1005500085060430870608000030850601308706CE
:100560000800003085062130870608000030850627
:10057000113087060800003085060830870608001D
:10058000003085061830870608003D18ED21BD189B
:10059000F9213D190522BD1911223D1A1D22BD1A4E
:1005A0002C223D1B3E22BD1B49225E185422DE1820
:1005B0005F225E196A22DE1978220800B601B301B3
:1005C000B4013C1CE62ABC01BC14E82ABC013C1462
:1005D0003C08B6006400EC2AED2AEE2AEF2AF02A45
:1005E000FF30B41B8500B41F8501B30BEA2AB40B9E
:1005F000EA2A0310B60CB608031DEA2A0030BB0035
:100600003C08BA00CB2108008F08031908008F01AD
:1006100078308E00C80F2E2DC80A441C342B461C7F
:10062000252BCA1C162BCA014A15422B4A1D1B2B0F
:10063000CA01CA15422BCA1D202BCA014A16422BD9
:100640004A1E422BCA01CA14422B4A1D2A2BCA0138
:100650004A16422BCA1D2F2BCA014A16422B4A1E8C
:10066000422BCA01CA14422BCA1C392BCA014A1593
:10067000422B4A1D3E2BCA01CA15422B4A1E422B51
:10068000CA014A15C41C692BC61C5A2BCB1C4B2B08
:10069000CB014B15772B4B1D502BCB01CB15772B5B
:1006A000CB1D552BCB014B16772B4B1E772BCB013C
:1006B000CB14772B4B1D5F2BCB014B16772BCB1D10
:1006C000642BCB014B16772B4B1E772BCB01CB1416
:1006D000772BCB1C6E2BCB014B15772B4B1D732B24
:1006E000CB01CB15772B4B1E772BCB014B15441D24
:1006F0009E2B461D8F2BCC1C802BCC014C15AC2B7C
:100700004C1D852BCC01CC15AC2BCC1D8A2BCC01E0
:100710004C16AC2B4C1EAC2BCC01CC14AC2B4C1D72
:10072000942BCC014C16AC2BCC1D992BCC014C1628
:10073000AC2B4C1EAC2BCC01CC14AC2BCC1CA32B67
:10074000CC014C15AC2B4C1DA82BCC01CC15AC2BE3
:100750004C1EAC2BCC014C15C41DD42BC61DC52B77
:10076000CD1CB62BCD014D155F13E22B4D1DBB2BC0
:10077000CD01CD15E22BCD1DC02BCD014D16E22BA9
:100780004D1EE22BCD01CD14E22B4D1DCA2BCD0108
:100790004D16E22BCD1DCF2BCD014D16E22B4D1E5C
:1007A000E22BCD01CD14E22BCD1CD92BCD014D1563
:1007B000E22B4D1DDE2BCD01CD15E22B4D1EE22B84
:1007C000CD014D155F1B0B2C441E0B2C461EFC2B24
:1007D000CE1CED2BCE014E15192C4E1DF22BCE0149
:1007E000CE15192CCE1DF72BCE014E16192C4E1EF0
:1007F000192CCE01CE14192C4E1D012CCE014E16F3
:10080000192CCE1D062CCE014E16192C4E1E192C5D
:10081000CE01CE14192CCE1C102CCE014E15192C45
:100820004E1D152CCE01CE15192C4E1E192CCE01A5
:100830004E15C51D402CC71D312CCF1C222CCF01BD
:100840004F154E2C4F1D272CCF01CF154E2CCF1DF1
:100850002C2CCF014F164E2C4F1E4E2CCF01CF14F7
:100860004E2C4F1D362CCF014F164E2CCF1D3B2C3E
:10087000CF014F164E2C4F1E4E2CCF01CF144E2CB5
:10088000CF1C452CCF014F154E2C4F1D4A2CCF01AC
:10089000CF154E2C4F1E4E2CCF014F15451E752CDB
:1008A000471E662CD01C572CD0015015832C501D90
:1008B0005C2CD001D015832CD01D612CD00150169A
:1008C000832C501E832CD001D014832C501D6B2CF4
:1008D000D0015016832CD01D702CD0015016832CC3
:1008E000501E832CD001D014832CD01C7A2CD00124
:1008F0005015832C501D7F2CD001D015832C501EF9
:10090000832CD0015015C51EAA2CC71E9B2CD11CB0
:100910008C2CD1015115B82C511D912CD101D11520
:10092000B82CD11D962CD1015116B82C511EB82CC3
:10093000D101D114B82C511DA02CD1015116B82CC5
:10094000D11DA52CD1015116B82C511EB82CD101A6
:10095000D114B82CD11CAF2CD1015115B82C511D7C
:10096000B42CD101D115B82C511EB82CD101511580
:10097000451FE02C471FD12CD21CC22CD20152158E
:10098000DF13EE2C521DC72CD201D215EE2CD21D36
:10099000CC2CD2015216EE2C521EEE2CD201D214C7
:1009A000EE2C521DD62CD2015216EE2CD21DDB2C71
:1009B000D2015216EE2C521EEE2CD201D214EE2C85
:1009C000D21CE52CD2015215EE2C521DEA2CD2017C
:1009D000D215EE2C521EEE2CD2015215DF1B172D14
:1009E000C51F172DC71F082DD31CF92CD301531574
:1009F000252D531DFE2CD301D315252DD31D032DDD
:100A0000D3015316252D531E252DD301D314252D87
:100A1000531D0D2DD3015316252DD31D122DD3019A
:100A20005316252D531E252DD301D314252DD31C4C
:100A30001C2DD3015315252D531D212DD301D31565
:100A4000252D531E252DD3015315BD214008C4006B
:100A50004108C5005F18DF145F1CDF104808C9009B
:100A60000C304A05031D05120C304B05031D851281
:100A70000C304C05031D05100C304D05031D851071
:100A80000C304E05031D87100C304F05031D071158
:100A90000C305005031D07100C305105031D871243
:100AA0000C305205031D07120C305305031D87112E
:100AB00049080E020318882D12304A05031D051639
:100AC00012304B05031D851612304C05031D05140D
:100AD00012304D05031D851412304E05031D871479
:100AE00012304F05031D071512305005031D071462
:100AF00012305105031D871612305205031D0716CB
:100B000012305305031D8715FF30480203190800F2
:100B10008F08031D0800982049080E02031C882D29
:100B200018304A05031D051206304A05031D051637
:100B300018304B05031D851206304B05031D851625
:100B400018304C05031D051006304C05031D051417
:100B500018304D05031D851006304D05031D851405
:100B600018304E05031D871006304E05031D8714EF
:100B700018304F05031D071106304F05031D0715DB
:100B800018305005031D071006305005031D0714CB
:100B900018305105031D871206305105031D8716B5
:100BA00018305205031D071206305205031D0716A3
:100BB00018305305031D871106305305031D871593
:020BC00008002B
:084000000300030003000900A6
:02400E00CC33B1
:10420000010078007A007C007E007B0079007F004E
:104210007D007A0078007E007C007D007F00FF003A
:104220000200F200F600FA00FE00F200F600FA00CA
:10423000FE00F200F600FA00FE00F200F600FF00B9
:10424000FF00050005000500050009000900090040
:1042500009000D000D000D000D0011001100FF0000
:104260000100FF00FF00FF00FF00FF00FF00FF0054
:10427000FF00FF00FF00FF00FF00FF00FF00FF0046
:10428000FF00FF00FF00FF00FF00FF00FF00FF0036
:10429000FF00FF00FF00FF00FF00FF00FF00FF0026
:1042A000FF00FF00FF00FF00FF00FF00FF00FF0016
:1042B000FF00FF00FF00FF00FF00FF00FF00FF0006
:1042C000FF00FF00FF00FF00FF00FF00FF00FF00F6
:1042D000FF00FF00FF00FF00FF00FF00FF00FF00E6
:1042E000FF00FF00FF00FF00FF00FF00FF00FF00D6
:1042F000FF00FF00FF00FF00FF00FF00FF00DD00E8
:00000001FF
